:020000040000FA
:100000008A150A125B290000F20003088301A00090
:100010000A08A1000408A2000B1900000B18000038
:100020008B180000831203138A110A128C196020A6
:100030000C1B00008C1A00000C1A00000C190000A8
:100040008C1800000C1800000D1800008301220815
:10005000840021088A0020088300F20E720E090035
:1000C000831603171008110583128A110A120319E7
:1000D0008528AB008A110A122B19CF208A110A1227
:1000E0002B1889208A110A12AB19DB208A110A12F7
:1000F000AB1ABB208A110A12AB18C2208A110A124D
:100100002B1AAF208A110A126028831203138C1154
:100110000800AC01C4018316901190119011901148
:100120000830A100B830A2008830A000C030A6007E
:100130000830A40096019001831203138C118316DA
:100140000317063098003B309100FF3093000130D8
:10015000970083120130AD000313031708008316C4
:1001600011121012101111159514831203138C1112
:1001700003174414080083169012831203138C1182
:1001800003170800831690101208130592018312BA
:1001900003138C110317B000831203170800831692
:1001A00011111011101211169510831203138C11D6
:1001B0000317C40108008317831603171408A03E11
:1001C000840083120008A000840A0008A100840AA9
:1001D0000008A2008316031714089011831203135A
:1001E0008C110317C50020083C39B100243A8A114C
:1001F0000A12031928293108043A8A110A1203192C
:1002000008293108343A8A110A1203198A29080088
:1002100045088A110A12031D1D292E08213A8A1148
:100220000A12031D132983160830A1008830A0008C
:100230008A110A12831282290800083A8A110A12C6
:10024000031D232908004508103A03190800080077
:10025000450818398A110A12031D7B292E08063A0F
:100260008A110A12031D38298A110A127E247A295A
:100270002E08663A8A110A12031D44298A110A12AD
:100280007E248A110A127A292E08053A8A110A1246
:10029000031D50298A110A127B238A110A127A2916
:1002A0002E08033A8A110A12031D59298A110A12CB
:1002B0007A292E08013A8A110A12031D7729270884
:1002C000013A8A110A12031D6B298316191483122D
:1002D0008A110A127A292708023A8A110A12031D82
:1002E0007A2983161A1483128A110A127A298A111A
:1002F0000A126A2D0800083A8A110A12031D812980
:100300000800080083160317A501C830A400831253
:10031000AE0108008317220884000008A300840AA5
:100320000008A400840A0008A500840A0008A600AA
:10033000840A0008A700840A0008A800840A0008AC
:10034000A900840A0008AA0083160830A100A400AE
:1003500083122308213A88300319C8308316A0007D
:1003600015128312AE0123088A110A120319E82913
:100370002308013A8A110A120319032A2308023AB0
:100380008A110A120319182A2308803A8A110A12BC
:100390000319242A2308813A8A110A120319362ADA
:1003A0002308823A8A110A120319482A230860395D
:1003B000203A8A110A120319AD2C23086039403AF9
:1003C0008A110A12031D0C2B8A110A12AC2C080088
:1003D0002408013A8A110A120319872B2408053AC6
:1003E0008A110A1203196F2B2408093A8A110A127A
:1003F00003191C2C2408033A8A110A120319CB2B67
:100400008A110A120C2B2408013A8A110A120319C4
:10041000C82B24080B3A8A110A1203196B2C2408E2
:10042000033A8A110A1203190C2C8A110A120C2B96
:100430002408013A8A110A120319922B2408033A5C
:100440008A110A120319D62B2408083A8A110A12B3
:1004500003190F2C2408063A8A110A120319522A8A
:100460002408003A8A110A120319112B24080A3AA7
:100470008A110A1203194D2C2408003A8A110A1213
:100480000319202B2408063A8A110A120319522A4A
:100490002408003A8A110A1203194B2B8A110A12F6
:1004A0000C2B08002608223A8A110A120319012D82
:1004B0002608213A8A110A1203194F2D02308A00A8
:1004C000031026080339673E03188A0A82000C2BA2
:1004D0006B2A852AB52A0630AE000830B500933065
:1004E000B2000530B3008A110A128D25B400AA08A3
:1004F0008A110A12031D802A29022908031CB4004C
:10050000B40A8A110A127E2408000630AE000310D5
:10051000250D8A110A127925B2000310250D013E1E
:100520007925B3000230B2070318B30A8A110A1200
:100530008D25B4000230B202031CB303AA088A114D
:100540000A120319A62A8A110A12AE2A34082902AD
:100550008A110A120318AE2A2908B4000830B5001F
:10056000B40A8A110A127E2408006630AE002708F9
:100570008A110A12031DC62A2808031DC62A3F3005
:10058000B2000630B3008A110A12FD2A0630B30009
:100590004130B200BB018A110A120326B20A2702B7
:1005A0008A110A12031DDC2A8A110A120326280264
:1005B0008A110A120319E82AB20ABB0A453032022C
:1005C0008A110A12031CCB2AAE018A110A120C2BC3
:1005D000063025028A110A12031CF22AAE018A1182
:1005E0000A120C2B250DB3003B088A110A120926AA
:1005F000B200B30A3B080926B3008A110A12032687
:10060000B40029022908031CB4000830B500B40A5C
:100610008A110A127E240800831603171814831205
:100620000800831626088400831283172D08800093
:10063000840A800183160230A500C830A400080097
:1006400083161708023A8A110A12031D2D2B8312F2
:1006500027088A110A12031D2D2B83161708033A47
:100660008A110A12031D0C2B83122708003C8A11E1
:100670000A12031C0C2B2708383E8400831700083D
:10068000F000831626088400700880000230A50060
:10069000C830A40008000F302705013A8A110A1259
:1006A0000319602B0F302705023A8A110A12031D25
:1006B0000C2B031083161A1803148A110A12642BC8
:1006C0000310831619180314260884008001800D76
:1006D000840A80010230A500C830A4000800250863
:1006E000AF008A110A12AF1B0C2B8A110A12822149
:1006F0000530AE000800AE01AC012F08831696004D
:100700008A110A120319862B023097000800250867
:10071000013A8A110A12031D0C2BAD108A110A121C
:100720008221080025088A110A12031D0C2B2608B5
:10073000031D0C2B831603301705023A8A110A1287
:10074000031DAD2B83120F302705031DAD2B831620
:1007500018108A110A128221080083160330170527
:10076000033A8A110A12031D0C2B83120F3027053E
:10077000023C8A110A12031C0C2B83170F30270529
:100780008316983E840000108A110A128221080004
:100790008A110A120C2B2508013A8A110A12031D2C
:1007A0000C2BAD148A110A128221080025088A1127
:1007B0000A12031D0C2B2608031D0C2B8316033075
:1007C0001705023A8A110A12031DF12B83120F300A
:1007D0002705031DF12B831618148A110A12822192
:1007E0000800831603301705033A8A110A12031D05
:1007F0000C2B83120F302705023C8A110A12031CAE
:100800000C2B83170F3027058316983E84000014A5
:100810008A110A12822108008A110A120C2B8316EF
:1008200026088400831283172C0880008316013069
:10083000A500C830A40008002508013C8A110A124E
:10084000031C0C2B2508AC008A110A1203192B2C4F
:100850008316033097008A110A1282218316031728
:10086000C830AA000830A9008830A8000830AD00C0
:10087000D030AE004830AC00D830B2000830B10003
:100880008830B0000830B500D830B6004830B40029
:100890000E3099000E309A00080083161708033AAC
:1008A0008A110A12031D0C2B83122708003C8A119F
:1008B0000A12031C0C2B2708383E840083170008FB
:1008C000F000831626088400700880000130A5001F
:1008D000C830A40008008316170883120339033AAE
:1008E0008A110A12031D0C2B2708383E8400831737
:1008F000250880008A110A12822108008316031736
:1009000083172608840083120317B70137083502BE
:100910008A110A120319A02C8A110A12B40B932C03
:100920008A110A129F2C8A110A128D258000B70A9B
:10093000840A8A110A12B20F862CB30A862CAE01E1
:1009400037088316A5004030240640398838A400B3
:0A0950008A110A12080008000800CE
:06095A008A110A122308B5
:10096000213A0319D42C8A110A122308223A0319B6
:10097000712D8A110A122308233A0319712D8A1145
:100980000A122308A13A0319712D8A110A122308A9
:10099000A23A0319712D8A110A122308A33A0319E6
:1009A000712D8A110A120C2B2408013A8A110A129D
:1009B0000319712D2408023A8A110A120319712DA4
:1009C0002408033A8A110A120319712D2408063AE1
:1009D0008A110A120319012D2408093A8A110A12F0
:1009E0000319742D24080A3A8A110A120319712D69
:1009F00024080B3A8A110A120319712D8A110A125E
:100A00000C2B831203170630AE000830B500260801
:100A1000013A8A110A120319202D0310270D8A1199
:100A20000A128325B2000310270D013E8325B3006F
:100A30008A110A128D25B400B20A8A110A12402DB9
:100A40002608023A8A110A120319392D0310270DBC
:100A50008A110A128325B2000310270D013E832557
:100A6000B3008A110A128D25B400B20A8A110A1243
:100A7000402D2608033A8A110A1203190C2B08008C
:100A80002A088A110A12031D4A2D2908340229084E
:100A90000318B400B40A8A110A127E240800063032
:100AA000AE000830B500B730B2000530B3008A118F
:100AB0000A128D25B400AA088A110A12031D642D9A
:100AC00029022908031CB400B40A8A110A127E24E0
:100AD000080008008A110A122E08063A03197E241B
:100AE00008008A110A120C2B2130AE00831603175E
:100AF0000800F00005308A008130700703188A0A68
:100B00008200A5340534F00005308A008B30700770
:100B100003188A0A8200CE3405348312031733087F
:100B20008A00320882001234013400340134003467
:100B3000003400340834003400340234003400340B
:100B400000340234013400340134093402342934CD
:100B50000034013401340434803432340934043430
:100B600000340034023403340034003400340934D7
:100B7000213400340134003401342234343400345C
:100B80000734053481340334083400340A3407341C
:100B9000053401340334083400340A343434063460
:100BA000A034FF3409340134A1340134093402344F
:100BB000A13400340634A134FF3409340334093439
:100BC00004341534803425347F34353400344534CE
:100BD000FF347534083495340834813402340934D0
:100BE0000534093406341534803425347F343534E3
:100BF00000344534FF347534083495340834913466
:100C00000234C034C0348312031733088A00320818
:100C10008200F0000310F00D8A110A121C26B600A3
:100C2000F00A8A110A121C26F00070088A003608A1
:100C3000330703188A0A820006308A0023307007BF
:100C400003188A0A820027340634333406343F34CA
:100C5000063445340634613406347D340634893430
:100C60000634933406343F340634A3340634B734A0
:100C70000634E5340634F1340634FB3406340634E5
:100C8000033409340434043408341C340334493440
:100C900000344F340034433400346134003472344F
:100CA000003464340034533400342D3400344B3475
:100CB0000034653400347934003473340034203423
:100CC00000341C3403344D340034613400346E3449
:100CD000003475340034653400346C34003420340E
:100CE000003456340034653400346C3400346534D8
:100CF00000347A340034203400340C340334563455
:100D00000034313400342E34003430340034303484
:100D100000340A3403344334003466340034673416
:100D2000003431340034103403344E3400346F3422
:100D300000347434003468340034693400346E3460
:100D4000003467340034143403344D3400346934CF
:100D5000003463340034723400346F34003463344C
:100D600000346834003469340034703400342E3474
:100D70000334503400346934003463340034313483
:100D800000343634003443340034373400343634DD
:100D900000343534003420340034553400345334B6
:100DA00000344234003420340034493400344F34A9
:100DB0000034433400346134003472340034643419
:100DC000003473340034203400340C34033456348B
:100DD0000034313400342E340034303400343034B4
:100DE00000340A3403344334003466340034673446
:100DF000003431340034103403344E3400346F3452
:100E000000347434003468340034693400346E348F
:060E1000003467340034D9
:10100000030883120317C3000408BD0083160317E7
:101010008A150A12A81B3C28290883120317C1004D
:10102000C2008A150A1203192C28831603172A08EE
:1010300083120317BE0083173E0884000008F100E6
:101040003D088400C31F831371088000BD0ABE0AD7
:101050008A150A12C10B1B28831628084039403A0A
:101060008838A8000830A90083124208F10043081C
:1010700083007108031408008312031743088300D8
:1010800003100800030883120317C3000408BD00FF
:10109000831603178A150A12B01B7E2831088312A3
:1010A0000317C100C2008A150A1203196E2883169D
:1010B0000317320883120317BE0083173E0884000B
:1010C0000008F1003D088400C31F831371088000ED
:1010D000BD0ABE0A8A150A12C10B5D2883163008A4
:1010E0004039403A8838B0000830B10083124208D5
:1010F000F1004308830071080314080083120317EA
:101100004308830003100800F1000308831203174B
:10111000C30071080F39C1000408BE0041088316DE
:1011200003178A150A12AC1BBB28AD008A150A12D8
:101130000319AF282E088312BD008317C31F831322
:101140003E0884000008F10083173D088400710800
:101150008000BD0ABE0A8A150A12C10B9D2883169B
:101160002C084039403A8838AC00831203174308F2
:1011700083000314080003100800F1000308831221
:101180000317C30071080F39C1000408BE004108ED
:10119000831603178A150A12B41BF428B5008A15A2
:1011A0000A120319E82836088312BD008317C31FEB
:1011B00083133E0884000008F10083173D08840073
:1011C00071088000BD0ABE0A8A150A12C10BD62812
:1011D000831634084039403A8838B4008312031724
:1011E0004308830003140800031008008317033921
:1011F000983E84000014080083170339983E840049
:101200000010080083120317441C080083161011F5
:10121000111595146300000095101012111610118D
:101220001111080083120317AD1C080083169510D6
:10123000111610121111101115158312BB018030F7
:10124000BC008A150A12BB0B2329BC0B2329831669
:10125000151108008316031795118312BC01BB01F9
:101260008A150A12BB0F3229BC0F32298A150A12BD
:101270003A2108008316031797010130910090016D
:10128000083095008312AC010130AD00B801B901FE
:10129000BA01FF30AE00831203138C1183168C1534
:1012A0000B178B17080083160317951195149701D8
:0612B00003138C1108007D
:0A12B6001E30F200F20B5D298316D2
:1012C000031381178A150A123A21831603178A1508
:1012D0000A12640003301705033A031D69298312BB
:1012E0000313850186018701F8018A150A123C2241
:1012F0008A150A12831323308400083000208A15CF
:101300000A12031C86298A150A122A228312031341
:10131000F8088A150A12031978298A150A127B22FD
:101320008A150A125D228A150A12AD21831203134F
:101330008A150A12A308031978298A150A12831339
:101340008312031323308400083084208A150A1284
:10135000031C9D298A150A12782983120313013070
:10136000AC000830AB00233084002D30B8000130D1
:10137000F4000630F50074098312031385008A1502
:101380000A12F0210310F40D8A150A12F50BBB297D
:10139000FF3085000130F4000330F500740983123A
:1013A000031387008A150A12F0210310F40D8A1521
:1013B0000A12F50BCE29FF30870083120313BF30CA
:1013C00087008A150A12F021831203137F308700E9
:1013D0008A150A12F02183120313FF3087000800D8
:1013E0000608F6000830F70003100408B9003808B2
:1013F00084000008BA0039088400831203138A1598
:101400000A12AB080319152A8A150A12F61B142AA8
:101410008A150A12BA1F152ABA132C088000AB03CA
:10142000840A8A150A12152ABA170310AC0AF60D97
:101430000310BA0D03183A148A150A12F70BFD2986
:101440000408B900380884003A088000390884008C
:10145000B80A0800013083120313F8008A150A1233
:10146000A31F3B2AFF30AD00AE00AF00B000B100BB
:10147000B200B300B40008008316031300308500E7
:10148000FF308600003087008316031306309F006C
:1014900083120313FF308500870083160313811323
:1014A00083120313AC01FF30AD00AE00AF00B000FB
:1014B000B100B200B300B400080083120313A3010B
:1014C000A401A501A601A701A801A901AA0108007C
:1014D000FF3083120313F40000008A150A12F40B84
:1014E0006C2A0800831203130830F4008A150A12CC
:1014F000F40B762A0800FF30F400FF30F5000000FE
:1015000000008A150A12F50B7F2A8A150A12F40BBD
:041510007D2A080028
:044000000034003454
:02400E00FA3F77
:00000001FF
